:020000040000FA
:060000000219FD020310CD
:030013000204FFE5
:03001B0002008D53
:03002B000202D5F9
:03005B0002050E8D
:030073000202FD89
:100080000406080C10182030406080A0C0C2AFC227
:10009000A853E6EFC28E856B8BC0D0D2D3C0E0C030
:1000A000F0C2CAA8CCA9CDD2CAD2AF758A00C3E823
:1000B000956CF8E9956DF9C3E913F9E813F8E5666D
:1000C0006007C3E913F9E813F8E97025E8956E4075
:1000D00020956E501CE582B410177C007B007A00DE
:1000E0007908900000A86AE5667004C3E813F80177
:1000F000FA900000D2A8D2AA61BAE0FDC39CC398CE
:1001000040EF98EB33FB0582E0FCC39DC39840E1D0
:1001100098EB33FB0582E0FDC39CC39840D398EB7A
:1001200033FB0582E0FCC39DC39840C598EB33FBCD
:100130000582E0FDC39CC39840B798EB33FB058272
:10014000E0FCC39DC39840A998EB33FB0582E0FD1A
:10015000C39CC398409B98EB33FB0582E0FCC39D96
:10016000C398408D98EB33FB05822175900000D237
:10017000A8D2AA61BAE0FDC39CC39840EF98EA33C5
:10018000FA0582E0FCC39DC39840E198EA33FA0582
:1001900082E0FDC39CC39840D398EA33FA0582E01D
:1001A000FCC39DC39840C598EA33FA0582E0FDC3BD
:1001B0009CC39840B798EA33FA0582E0FCC39DC31C
:1001C0009840A998EA33FA0582E0FDC39CC39840A1
:1001D0009B98EA33FA0582E0FCC39DC398408D9852
:1001E000EA33FA0582EBC46B6A54F0F9EAC454F0BE
:1001F000C3996009900000D2A8D2AA61BAEBF4C4F6
:1002000054F0F9EAF4C4540F49FAEBF4C4540FFB68
:10021000C3EAF99460FAEB9400FB5020C3E97B0039
:100220007A0079006016C3135006F9C39552600A2C
:10023000E9F552755300790080020553303A27C31F
:10024000EA94D0F8EB9407F9400BE8FAE9FB203583
:1002500009D235415A303502C235203902B235C390
:10026000EA33FAEB33FBEB2B3B3BF9C3EB13FBEA33
:1002700013FAEA29FAEB3400FB30E3047AFF7BFF40
:10028000E5255403601B202A18E55D33F9EB700760
:10029000C3E99A4002E9FAE53CC4332AFAEB340098
:1002A000FBC3EA33C4540FF8EB33C454F048F8707E
:1002B00005EA60027801C3EB13FBEA13FA90000031
:1002C000D2A8D2AAE52260021522819E900000D217
:1002D000A8D2AA61BAC0D0C0E0C2CF0541E5236070
:1002E000021523C3E554600575550041F8E5552412
:1002F00001F55550037555FFD0E0D0D032C2AF5351
:10030000E67F7592FA7593FFC22053917FD2AF3288
:10031000C0E0E58A303408856B8BF0A3D0E032D0A2
:10032000E0C2AF53E6EFC0D0C0E0C0F0D2D3D2AF4E
:100330005388EFA88AA98C758A00758C00438810B1
:1003400030331FE8C4540FFAE9C454F04AFAC31317
:100350002AFAC3E833F8E933F9E82AFAE93403FB67
:1003600061AB30320FC3E833E933FAE82AFAE934F3
:1003700000FB61AB303115E875F056A4AAF0E975C1
:10038000F056A42AFAC5F03400FB61ABE875F02BF7
:10039000A4AAF0E975F02BA42AFAC5F03400C3131F
:1003A000FBEA13FAC3EB13FBEA13FAC3EB9409500D
:1003B00009C3EA949AEB940350160522E5227002D1
:1003C0001522C3E5229432500281F275540081F562
:1003D000E522600215223036067C007D0461EAAC1D
:1003E00031AD32303A04AC33AD34C3EA9CFAEB9D04
:1003F000FB9208AE60AF61303A425007203509D217
:10040000358108303502C235303504AE62AF632025
:100410003902B235C3EA33FAEB33FBA208500AEAD9
:10042000F42401FAEBF43400FBC3EA9428FAEB94C9
:1004300000FB501478007A007B008148A208500825
:1004400078007A007B00819EE52554036019202AFC
:1004500016E55DF9EB7007C3E99A4002E9FAE53C5D
:10046000C42AFAEB3400FBEA8EF0A4F9AAF0EB8E72
:10047000F0A42AFAC5F03400FBC3EB13FDEA13F82D
:100480000FEF146004C3E833F8C3E933EA33FAEB3F
:1004900033FBDFEDEB30E20678FF7AFF7B03885415
:1004A000D230E86003755500C3E55BFC955C400203
:1004B000AC5CC3EC95545008EC75F004A4FAABF0B6
:1004C000EAF4F8EBF45403F9C3E8940AFAE9940067
:1004D000FB50047A007B00885689578A588B5975DF
:1004E000230AD0F0D0E0D0D053F7DF43F74043E603
:1004F000103275230AD0F0D0E0D0D043E61032C2DB
:10050000AAD28EC2CA85CC6C85CD6DD2CA32C2AF9A
:10051000C0D0C0E0D2D3A8F9E55A30E10AE5FA200C
:10052000E13520E032A12FE5FA30E12B20E028C3AD
:10053000E55713F8E55613F5FB88FCC3E55913F8A6
:10054000E55813F5E988EA85575A53F7BFD2A83022
:100550003402D2AA53E6EF53F7DFD0E0D0D0D2AFC7
:10056000327901801479038010790A800C791E8019
:10057000087964800479C880007817E4D5E0FDD854
:10058000FAD9F62278FF20282879A1E76023E548E8
:10059000601F74FF8548F084853FF030290375F0B3
:1005A00005A4F8C5F0600278FFC3E8955D5002A885
:1005B0005D885C22C3E54794E4E5489400E55C501F
:1005C0000314A1C5046002F55C2275E89022055E63
:1005D000C3E55E9408405330EDF4A8BDA9BE755E36
:1005E00000E9FA79A0E76041EA7006E55F601880EB
:1005F0000CC3E8955F600EE55F5005600A14800744
:100600000460FA8002E55FF55FC39569401B755B86
:10061000C0C394044013755B80C39404400B755BA6
:1006200040C394044003755B0022E55B2410500234
:1006300074FFF55B22743279A687F0A4C5F0A2F7A7
:1006400033F55D227547007548F022C2AFC2CAA8D3
:10065000CCA9CDAA4130CF010AD2CAD2AFAB42ACAD
:100660004388428943C3E89BF8E99C202808F93075
:100670002C02E15BC1B4AD448A44F9EA9DFA6006FC
:1006800078FF79FFC199AE45AF468B458C46A842AD
:10069000A943C3E89EF8E99FF9C3E54813FBE54782
:1006A00013FAE82AF547E93BF54850067547FF7508
:1006B00048FFE101AA47AB48AC47AD487E047F0242
:1006C000C3EB9404400D1E1FC3EB94084005202982
:1006D000021E1FC3ED13FDEC13FCDEF7C3EA9CFA08
:1006E000EB9DFBEF6009C3E913F9E813F8DFF7EAC4
:1006F00028FAEB39FB8A478B4850067BFF8B478BE8
:1007000048C3EB94025002D22C3028047F03E12C22
:100710007892E6FFC3E53D948240110FC3E53D9416
:10072000A040010FC3EF940640027F057E02E5481A
:10073000C4540FF9E548C454F0F8E547C4540F28F1
:10074000F8C3E89EFAE99400FB4009C3EA9401EB80
:10075000940050047A01E4FB0207A7AA47AB48EBD8
:10076000C4FEEAC4540F4EFCC3EA9CFAEB9400FBAF
:10077000C3E813C313F8EA28FAEB3400FB8A478B6B
:1007800048C3EB94024002C22C7802EBC4FE7B000B
:10079000EAC4540F4EFAC3EA98FA4005C3940150D4
:1007A000027A017892E6FF302002E1A7854E928519
:1007B0004F93D22043E680C3E49AF8E49BF9302CAF
:1007C00003020835E8FAE9FBD3E913FDE813FC88D6
:1007D0004E894FC3EF94036038EF20E00CE82CF80B
:1007E000E93DF9ECFAEDFB8013E828F8E939F9C3A3
:1007F000E82401F8E93400F97AFF7BFFC3EF9403A2
:10080000400F8A508B51884A894B8C4C8D4D020881
:100810006A885089518A4A8B4B8C4C8D4D302812F6
:100820007550F07551FF754CF0754DFF754EF075B4
:100830004FFF02086AE8FAD3E813FC884EC3EF942E
:10084000036021EF20E007E82CF8ECFA0155E828D6
:100850002401F87AFFC3EF940340098A50884A8C38
:100860004C02086A88508A4A8C4C302002016A7512
:100870003A02D22043E680E52554036034A847A914
:1008800048C3E913F9E813F8C3E913F9E813F8309A
:100890002804E92440F9C2AF53E67F759100C3E410
:1008A00098F594E499F595759104D22043E680D2A9
:1008B000AF22D221754900752000302B03752040EE
:1008C00001D0D221754900752040302B03752000DE
:1008D00078017901202C20E52554036002C221799A
:1008E00014E548C313700104F8C39414400278144B
:1008F000302804781B791B202010E549600C302833
:1009000003D53A04D222217811720549E59BF454AB
:1009100040B52002216230280908C3E89940011837
:1009200001F720210A08C3E899400201D001F7C26B
:100930002153E67F759100302C117594007595F860
:10094000759104D22043E6800208D0E5487EFFC3BB
:10095000334005C3334001FEC3E49E759400F59512
:100960002140C3E5399401500201D030210201D069
:10097000D802217601F7C222C2AF53E67F759100FB
:10098000855094855195759104854A92854B93D2F3
:100990002043E680D2AFE5255403600720290205F5
:1009A00039801030220D202B0A2021071581158156
:1009B0000213552278003021027801E53D75F007D9
:1009C000A4F9E5F028F5F0E9A2F013A2F113A2F2E0
:1009D00013F53DC394785003753D78C3E53D953ECE
:1009E0004009C290C292C29475D53F30200221EBDB
:1009F000854C92854D93D22043E68022203810C248
:100A0000AFD293C29175D50FD2AF759F0341CCC2BF
:100A1000AFD293C29575D53CD2AF759F0341CC2020
:100A20003810C2AFC29475D533C291D2AF759F133F
:100A300041CCC2AFC29075D533C295D2AF759F235A
:100A400041CC203810C2AFD291C29575D533D2AF08
:100A5000759F238077C2AFD295C29175D533D2AF3F
:100A6000759F138067203810C2AFC29275D53CC203
:100A700095D2AF759F038054C2AFC29275D50FC295
:100A800091D2AF759F038044203810C2AFD295C277
:100A90009375D53CD2AF759F138031C2AFD291C24E
:100AA0009375D50FD2AF759F238021203810C2AF28
:100AB000C29075D50FC293D2AF759F23800EC2AF7F
:100AC000C29475D53CC293D2AF759F13227A147B22
:100AD0007880127A107B8C800C7A0D7BB480067A39
:100AE0000B7BC88000E564D5E001227902E4D29353
:100AF000D5E0FDD292D5E0FDC292D5E0FDC293D5FE
:100B0000E0FDE920E002D29030E002D294E564D525
:100B1000E0FDE920E002C29030E002C2947496D574
:100B2000E0FDD9C9EAF8D5E0FDD8FBDBB8D29322C5
:100B3000C290C292C294D291D293D29575D53F22DF
:100B4000788076FF0876FF0876FF0876FF0876FF44
:100B50000876FF0876090876FF087601788C76011A
:100B60000876FF0876FF0876FF0876FF0876FF080C
:100B700076030876FF0876FF0876FF087625087664
:100B8000D00876280876500876040876FF087602A2
:100B90000876FF08767A0876FF0876070876010857
:100BA00076FF0876FF08760008760022FA75F00CCA
:100BB000A4ABF0EAC333F8740133F9E8C333F8E9BE
:100BC00033F9E8C32BF8E93400F9227888E6C394B6
:100BD00003D23A5002C23AC238E630E102D238A219
:100BE0003892397886E6149000809378A6F6788655
:100BF000E6F53FC394025003753F02789CE6753ECC
:100C0000FFB40203753EA0B40303753E8278A0E6EC
:100C1000F8600674282409D8FCF5697896E671AC6A
:100C200088318932789EE671AC883389347897E6CA
:100C300071AC883589367130223036117A007B00EC
:100C40007CFF7D007E00919F8B618A6022303A227A
:100C50007896E6FA7B00789EE6FC7D00C3EA33FADC
:100C6000EB33FBC3EC33FCED33FD7E0A919F8B63CA
:100C70008A627896303A02789EE6FA7B007897E6A8
:100C8000FC7D007E00303A10C3EA33FAEB33FBC33D
:100C9000EC33FCED33FD7E0A919F8B618A6022C3A9
:100CA000EC9EFCED9400FDC3EC9AFCED9BFDC3ECC7
:100CB0009423ED940050047C237D00C3EC94FFED5D
:100CC000940140047CFF7D017BFF0B7A000AEA70EF
:100CD00009C3EC33FCED33FD81CAEC8AF0A4AEF01D
:100CE000ED8AF0A42E947C40E4EAF460DD22D23652
:100CF000913912056D12056D7A007B007C1012058A
:100D000065E5542AFA74003BFBDCF37C04C3EB1367
:100D1000FBEA13FADCF7FFEB60027FFFC236913982
:100D20002278A5E6F954037000E9540C7000E954E8
:100D3000307000E954C07000227567007568007556
:100D400097DE7597AD7581C043FF8075EF0675A975
:100D50000071307580FF75F1F075A4007580FF7526
:100D6000D4FF75902A75F23F75A53F75902A75D509
:100D70003F75A60175E34075E2027130E4F8F6D8DC
:100D8000FD714012138B78988664753001C2AF12E2
:100D9000057551CD12056D51D312056D51D912054E
:100DA0006DB121C2AF75670075680078FA79FA30C5
:100DB0008507D9FBD8F7021C0071CB91397898864A
:100DC00064713075E405758811758E04758909752F
:100DD000C80475910475D84075D90875F781759E5A
:100DE0000375960075DA4275DB4275A82175E690A9
:100DF00075B801759B80759D0075D10C75BC5975D2
:100E0000BB1075E88075B201120561D2AF753C0068
:100E1000C230120575C231C232C233C234755200BB
:100E2000755300752200120571C3E522940A500221
:100E3000C1FAD231752200120571C3E522940A501D
:100E400002C1FAC231D232752200120571C3E52205
:100E5000940A5002C1FA75E4D5758851758E0175F2
:100E600089AA758C00758D00C2A9D2ABD2AA756B08
:100E7000C0756A14756E50C232D23475220A1205DA
:100E800071756A10C3E522940A75520075530040CB
:100E900069758E0C756B80756A28756E2875220AC7
:100EA000120571756A20C3E522940A7552007553C4
:100EB000004047758E0C756BC0756A14756E14759D
:100EC000220A120571756A10C3E522940A75520050
:100ED000755300402575E405758811758E04758974
:100EE00009D2A9C2ABC2AAC234D2337522001205FC
:100EF00071C3E522940A4002A1A3120565203003C4
:100F0000020DA3C2AF51CD51CD51CDD2AF12057557
:100F1000203403303A03020FB8120565788CE6C31B
:100F200094015002E1B8E530C394015002E1B87574
:100F300067A57568F17F02D2369139120571C2AF8B
:100F4000C2369139C3E554947FD2AF406B1205612C
:100F5000C2AF51DFD2AFDFDF91EEC3EF7897F61269
:100F600005751214787F0AD2369139120571C2AF15
:100F7000C2369139C3E554947FD2AF50E81205616F
:100F8000C2AF51CD12056951CDD2AFDFDA91EEEF8C
:100F900024037896F6F87997E7C394234003985092
:100FA00006E824237897F61205751213D21214A7B7
:100FB0001205719139020DA375670075680012055D
:100FC00071C3E55494014002E110C2AF51DF51DF1B
:100FD00051DFD2AF120575753000E4F537F53805ED
:100FE00037E537F4703F0538789AE67819146012BF
:100FF000783214600D787D14600878FA14600375F7
:101000003800C3E53898401D120B301205611538C1
:1010100075370078998664C2AF120ADFD2AF78982C
:101020008664120571120569E5237003020DA3C3DE
:10103000E5549401500AC3E55294015016020FDFA3
:10104000120571E5237003020DA37552007553005C
:101050000211F5C3E55294017017C2AF120B30783C
:10106000998664120ACD78988664D2AF12057121F0
:10107000E7C3E55294027017C2AF120B307899861D
:1010800064120AD378988664D2AF12057121E7C33F
:10109000E55294037017C2AF120B30789986641230
:1010A0000AD978988664D2AF12057121E7C3E55258
:1010B00094047017C2AF120B3078998664120ADF5D
:1010C00078988664D2AF12057121E7C3E552940582
:1010D0007017C2AF120B3078998664120ADF7898C5
:1010E0008664D2AF12057121E7C3E55294077019E7
:1010F000C3E55394065002012F7401303A02740381
:101100007888F6C238C23921E7C3E55294087019CD
:10111000C3E55394065002012F7402303A0274045E
:101120007888F6D238D23921E7C3E552940970178E
:10113000C3E55394065002012F303A0BC37888E67A
:101140009402F6C23A21E7C3E552940A7016C3E549
:101150005394065002012F203A0A7888E62402F6BA
:10116000D23A21E7C3E55294147025C3E55394069F
:101170005002012FC2AF901A0B740093D2AF78883F
:10118000F613C238C2394002D2384002D2398057F1
:10119000C3E55294157038C3E5539406404FC2AF6F
:1011A000901A0B740093D2AFF8B801027402B8021F
:1011B000027401B803027404B8040274037888F658
:1011C00013C238C2394002D2384002D2398018C323
:1011D000E552940C70117567A57568F1C3E55394D9
:1011E00006400A71D2D2AF75520075530075670080
:1011F000756800012FC2AF120B30E4D2AFE4F55E88
:10120000F524F525F53D755E081205611205CA3015
:10121000EDFDA8BDA9BEE97001F8885F1205CE7585
:101220005E08C2AF120635855D5B855D5CD2AF306E
:101230003A07C238303502D238D228753900120A3E
:1012400088120AAB12064412064B12064412064BD1
:101250001206441208C21209B41209FC12064B12FB
:1012600008B2202C03120584302C031205B4120995
:10127000B4120A1F12064B1208C21209B4120A4213
:1012800012064B1208B21209B4120A6512064B126A
:1012900008C21209B4120A8812064B1205CA1208B3
:1012A000B21209B4120AAB1205CE12064B3028272F
:1012B000855D5B79187A0CC3E53999400EC228D256
:1012C000298A3B855D5B855D5C800CC3E554940198
:1012D0004003021253615D30291F202B1CE53B1493
:1012E0007006C229D22A4153F53B203A07C3E55480
:1012F000940140030212538064753C00203A0F7839
:10130000FA79A4E760027803C3E55598504FE523C6
:10131000604B303A17203805203507800F303502F2
:10132000800A202B07D22B855D5B418378F0302B20
:1013300005855D5B7820C3E5489850030212533061
:101340002B1BC22BC238303502D238D229753B1242
:10135000855D5B4153053CE55460026160753C006E
:10136000C2AF120B30752400752500D2AF12057183
:10137000120B3078A4E66006C291C293C295C3E511
:101380003C94044003020DA3020FDA901A0D78205A
:10139000910BE520B4550AA3910BE520B4AA028075
:1013A000137567A57568F1120B4071D275670075EA
:1013B0006800801D901A0378807B0A910BA308DBDC
:1013C000FA901A0F788C7B1A910BA308DBFA901A0B
:1013D0002922C2AF914E912B901A0074109110A344
:1013E00074079110A374219110901A0378807B0ADE
:1013F000910FA308DBFA901A0F788C7B1A910FA338
:1014000008DBFA9161913F901A2922E493F622E6D3
:10141000438F01538FFDFFC3E583941C400122EFEE
:101420008567B78568B7F0538FFE22438F02438FDD
:10143000018567B78568B7901A0DF0538FFC22902D
:101440001A0D74559110901A0E74AA9110227A30C8
:1014500079D07820901A40910BE520F709A3DAF7AC
:10146000227A3079D0901A40E7911009A3DAF92254
:101470007C05120575DCFB22C2AF120ACD120AD31D
:10148000120AD9120ADF120569120ACD120AD31202
:101490000AD9120ADF120569120ACD120AD3120AFA
:1014A000D9120ADFD2AF22C2AF120ADF120AD91252
:1014B0000AD3120ACD120569120ADF120AD9120ADA
:1014C000D3120ACD120569120ADF120AD9120AD301
:0614D000120ACDD2AF228A
:1019FD00020D39100721FFFFFFFFFFFF09FF01FF58
:101A0D0055AA01FFFFFFFFFF03FFFFFF25D0285061
:0D1A1D0004FF02FF7AFF0701FFFF0000FF3A
:101A4000234F5F4C5F313023202020202020202096
:101A500023424C48454C492445464D3842313023B9
:101A60002020202020202020202020202020202076
:101C0000C2AFC2D37597DE7597AD7581C075A90057
:101C100043FF80752438752503B1DB7529A5752A26
:101C2000F143F12053A4DFD28575D4FF75E3407DE5
:101C3000FA780379E67C10752200752300901DE880
:101C40007B0675249875250130850281482085081A
:101C5000D8FBD9F9DCF781BA308508D8FBD9F9DC93
:101C6000F781BAB19BE493A3C39A6004DDC381BA40
:101C7000DBDBB18D600281317B08E493FAA3B16EA6
:101C8000DBF87A30B16E752200752300B18DEAFC65
:101C9000EBFDC3ED94FE400EB18D8A278B28ED300D
:101CA000E0048A828B83B18D7AC270D8C3ED94FE32
:101CB000601950CEBD0029EC600F7520007521FF22
:101CC000752900752A000200008100A827A92808AC
:101CD00009D804D90281DDB191EAF281D10D81A642
:101CE000C3ED94035051EDA2E092007AC5C3E582A2
:101CF0009400E583941C508C200010438F02438F86
:101D0000018529B7852AB7F0300027A827A9280818
:101D100009438F01538FFDD804D902A132C3E58353
:101D2000941C4003A3A117E28529B7852AB7F0A325
:101D3000A117538FFC81827AC1BD030CE493A3FAEF
:101D4000B152DCF8B14A81828184AA22AB23B16E00
:101D5000EBFAEA6222752608C3E52313F523E52290
:101D600013F52250066323A0632201D526EAB1DBD6
:101D7000B1DB75260AEAF4200102D285300102C2E5
:101D800085B1DBC3134002C201D526EB22B191EA33
:101D9000FB208502A191308502A196752608AE240C
:101DA000AF25C3EF13FFEE13FEB1DFB1DBC3EA13C0
:101DB0003085024480FA30E703632201C3E5231330
:101DC000F523E52213F52250066323A0632201D5F3
:101DD00026D9E52265236523F52222AE24AF250E00
:101DE0000FDEFEDFFCD20122424C48656C693437BD
:061DF0003164E8B10601B8
:00000001FF
